:10000000E5C0FFC075C2FDC0FCC0FBC0FAC0F9C0AE
:1000100001C3F7C0F6C0F5C073C3F3C0F2C0FDCC96
:10002000E6CCA9CDB4CDBECD18CE2FCE00000000B9
:10003000A60EF9154C1DF22B3E498A6601020304F7
:10004000050607030303030414E6FF0000005AFF3C
:10005000FFFF000046FF1EFF000050FF1EFF0000D4
:1000600019FFFFFFFF00256E183F96FFFFFF0000FE
:10007000000000468CFF146EFFFFFF0000000738F1
:1000800089FF1E78FFFF0000000050FF1EFFFF00E9
:10009000000050FF78FF000046FFFF0000FF00FF58
:1000A0000000000000000000000000000000000050
:1000B0000000000000000000000000000000000040
:1000C0000000000000000000000000000000000030
:1000D0000000000000000000000000000000000020
:1000E00000020304050708090B0C0E0F1112141669
:1000F00017191B1D1E20222426282A2C2F313335A8
:10010000383A3C3F424447494C4F5255575A5D603C
:1001100064676A6D7174777B7E8286898D9195990B
:100120009DA1A5A9ADB2B6BABFC4C8CDD2D6DBE0F9
:10013000E5EAEFF4FAFF03030304040405050606E9
:100140000708090A0B0C0D0E0F11121416181A1CB1
:100150001E212326292C2F33363A3E42464A4F533E
:10016000585D63686E747A80878E959CA4ACB4BC2D
:10017000C4CDD6DFE9F3FDFFFFFFFFFFFFFFFFFF69
:10018000FFFFFFFFFFFFFFFFFFFFFFFFFFFFFFFF7F
:10019000FFFFFFFFFFFFFFFFFFFFFFFFFFFFFFFF6F
:1001A000FFFFFFFFFFFFFFFFFFFFFFFFFFFFFFFF5F
:1001B000FFFFFFFFFFFFFFFFFFFFFFFFFFFFFFFF4F
:1001C000FFFFFFFFFFFFFFFFFFFFFF0011241FBE28
:1001D000CFE5D2E0DEBFCDBF10E0A0E6B0E0E8E6BC
:1001E000FDE102C005900D92A23AB107D9F720E0D7
:1001F000A2EAB0E001C01D92A13FB207E1F7E3D649
:10020000B1CDFECE20ED37E0019720F0F901319716
:10021000F1F7FACF089590916400992349F088236B
:1002200021F083E187BBC49A089583E087BBC4981B
:100230000895815090E0FC01EA5CFE4F2491FC019E
:10024000E056FF4F849188BD29BD8091EB00882343
:1002500011F080E0E0CF0895CF93DF931F92CDB7E8
:10026000DEB79FEF98BD90E06983CCDF18BC698151
:10027000862F90E00F90DF91CF91C4CF811108C0FD
:1002800018BC19BC8091EB00882319F081E0C3CF22
:10029000D0CF089580916B008093BF0010926B00C7
:1002A0001092F0008BE58093C10080E0B4CF809184
:1002B000BF0080936B001092CC0080916B0088236C
:1002C00019F01092C10008958091C0008093C10080
:1002D0000895EF92FF920F931F93CF93DF93C82F50
:1002E0008B017B01EE0CFF1CEE0CFF1CD8E2CC2333
:1002F00071F081E090DF18BCD9BDC80183DF80E0D8
:100300008ADF18BC19BCC7017DDFC150F0CFDF9177
:10031000CF911F910F91FF90EF9008951F93CF936E
:10032000DF93C82FD62F18E2CC2301F18091C100B2
:100330008D131CC081E06FDF80916400882321F061
:100340008091CE00811102C018BC19BD8AEF90E0E7
:1003500059DF80E060DF18BC19BC87E791E052DF0D
:100360008091C1008D1302C0C150DECFDF91CF91CB
:100370001F9108951F93CF93DF93D62F6AE0B7DCC8
:10038000192F6D2FCBDFC091C100CD1310C080E2BB
:1003900093E038DF6C2F812FC1DF8091C1008C1377
:1003A00006C080ED97E0DF91CF911F912BCFDF91B9
:1003B000CF911F910895EF92FF920F931F93CF93C8
:1003C000863018F006E910E002C00AEF10E078016C
:1003D000EE0CFF1CC82FCC23D1F018BC19BCC801EF
:1003E00011DF81E018DF80916B00882321F080917C
:1003F000DF0044DF06C08091DC009091DE0098BDF4
:1004000089BDC701FFDE80E006DFC150E4CFCF9198
:100410001F910F91FF90EF900895EF92FF920F932D
:100420001F93CF938C017C01F594E794C62FCC23C6
:1004300051F081E0F0DEC801E5DE80E0ECDEC701CE
:10044000E1DEC150F4CFCF911F910F91FF90EF905B
:100450000895CF93C82F68E270E082E03ADF80EF22
:1004600090E0D0DE64E670E08C2F33DF1092C200A3
:10047000CF91089586B383FB882780F991E0982770
:100480008091AA00880F892B8093AA009091A900DF
:10049000992311F08F7001C081708093A900809121
:1004A000A90090E008958091C100803120F48091EE
:1004B000C1008093C0008091C1008F5F8093C10014
:1004C0009091DD00891710F01092C100089580917D
:1004D000C1008093C0008091C100811103C0809150
:1004E000DD0002C08091C10081508093C100089559
:1004F00018958EBB6DBB84E28CBB86E28CBBE19908
:10050000FECF0895CF93DF932091C10080916700C3
:1005100090916B00880F880F880F97959927979572
:10052000692F682B622B6093EF002091D0003091EF
:10053000CF0090916A0080916900330F990F990F55
:10054000932B922B8295880F807E892B8093DB00E2
:100550004091CD0050916400309165009091CE00A3
:100560008091660070916800550F330F330F352B63
:10057000342B990F990F990F292F232B8295807F68
:10058000982F922B872F8295880F807E892B8093BE
:10059000ED00C091AB00D091AC00CE0104968F77F6
:1005A00099279093AC008093AB00A3DF8091AB00C0
:1005B0006091DB008F5F9DDF8091AB006091ED006B
:1005C0008E5F97DFCEBB84E18CBB86E18CBBE1996B
:1005D000FECF8C2F8F5F8EBB84E18CBB86E18CBB02
:1005E000E199FECF8C2F8E5F8EBB84E18CBB86E1C0
:1005F0008CBBE199FECFCD5FCEBB84E18CBB86E1A5
:100600008CBBE199FECF8091AB006DE58D5FDF91F2
:10061000CF916FCF1F920F920FB60F9211245F935D
:100620006F937F938F939F93AF93BF9364B175B193
:100630008091B000813021F5CB0196958795945D2E
:1006400062DB6D5F7F4F8091B2008823B9F08091AB
:10065000B20090E08617970728F48091B2008F5F70
:100660008093B2008091B20090E06817790740F45F
:100670008091B20081508093B20002C06093B200BA
:100680008091B0008330F9F4605171408091B100E5
:100690008823B9F08091B10090E08617970728F47D
:1006A0008091B1008F5F8093B1008091B10090E0A4
:1006B0006817790740F48091B10081508093B100B0
:1006C00002C06093B1008091B0008F5F8093B00052
:1006D000843010F01092B0008091B000823010F49D
:1006E0008CE001C08FE887B9BF91AF919F918F9146
:1006F0007F916F915F910F900FBE0F901F90189593
:100700001F920F920FB60F9211242F933F934F9386
:100710005F936F937F938F939F93AF93BF93EF9369
:10072000FF938091EE00882321F081508093EE00AA
:1007300039C48091AE009091AF00892B49F080912F
:10074000AE009091AF0001979093AF008093AE0000
:1007500091DE2091BD003091BE00892B09F4BAC111
:10076000203D87E0380730F42F5F3F4F3093BE00C5
:100770002093BD008091BD009091BE00823E24E098
:10078000920771F41092CC001092DF001092C10019
:100790001092CB0081E08093C6001092C50002C485
:1007A0003091C5002091B6003323B1F01092C20001
:1007B0002111F8C38332910521F48091C5008F5F28
:1007C00008C08634910509F0EDC381E08093B6003E
:1007D0008FE08093C500E6C3211171C120916B00A9
:1007E000222309F49DC0429708F49AC08091C60064
:1007F000811196C08091C700811192C08091C10083
:10080000803508F08DC08091CB00813009F459C04B
:1008100038F0823009F45DC0833009F464C080C0D0
:100820008091CC00811120C081E08093CB0087E1D2
:100830008093EA0080916A0018BC89BD8091EB002A
:10084000882311F080E0E7DC8FEF8093CC00809369
:10085000DF008091C800811104C08091CC0080939A
:10086000C8001092C9005CC08091C9009091CA0074
:10087000882329F09093CB001092C90004C085E032
:10088000891B8093CB008091CC00863921F493E0C2
:100890009093CB000AC08091CC008F3F51F482E04E
:1008A0008093CB0081E08093CC008093DF00C1DC9B
:1008B00037C08091CC00813099F582E08093CB00E5
:1008C0002FC08091EA0081508093EA00811128C0F6
:1008D000E6CF8093CA008091CC008639B0F4809135
:1008E000CC008F5F09C08093CA008091CC00823019
:1008F00060F08091CC0081508093CC008093DF0029
:100900008091CC008093C80008C084E08093CB0025
:1009100080E0B4DC87E090E075DC8091DF00AEDC45
:1009200080916B0081112CC08091BD009091BE0020
:10093000489731F58091C600811122C08091C10095
:10094000803140F48091D000882311F0ACDD18C0D4
:10095000BEDD16C08091C1008B3590F0E091F000B3
:10096000EE2351F0E150E093F000F0E0E356FF4F4A
:1009700080818093C10004C081E08093C70097DC30
:100980008091BD009091BE008434910509F068C04B
:1009900080916300813029F58091BC00823009F597
:1009A0008091B9009091BA000E97D8F480916B00B5
:1009B000882329F08091C600813009F051C010923F
:1009C000CC001092DF001092C1001092CB009091E9
:1009D000C60081E0282F291B2093C6008093C70002
:1009E0003FC08091C60081113BC08091BC00813026
:1009F00099F42091B9003091BA002E30310560F49D
:100A000090916B0091112CC090E59093C100809360
:100A1000C70018BC19BC24C08091C1008B3510F0F0
:100A200046DC1EC08091C100803569F41092C1007F
:100A300018BC19BC85E18093C5001092C30081E009
:100A40008093B6000DC080916B00811109C0809128
:100A50006800882329F08091C100803509F01ADCF4
:100A60008091C60081112BC080916B0081110FC055
:100A70008091BD009091BE00803A910541F4809133
:100A8000BC00823021F08091C100803559F4809102
:100A90006B008823A1F08091BD009091BE00843F3F
:100AA000914069F41092C1001092CC001092CB00DA
:100AB00018BC19BC81E08093C5001092C30010924D
:100AC000A8001092A70088E391E0909361008093C2
:100AD00060005EC21092B6008091C5008823A1F02C
:100AE0002115310559F02831310528F48091C300D2
:100AF0008F5F8093C3001092C20046C28091C200F3
:100B00008F5F8093C20040C22115310509F46AC18C
:100B100080916B00882309F4C8C01092CB00223169
:100B2000310508F0B6C08091BC008F5F8093BC0097
:100B30008091BC00813021F58091C1008093A60096
:100B40008091C100803138F48091CC00863919F44D
:100B50008FEF8093A6008091C100803541F0809195
:100B6000C100813521F08091C100823549F4109295
:100B7000C1001092CC001092DF0081E08093C7008A
:100B80008091A60090EB980F923090F49091BC0069
:100B9000923009F087C0803511F481E501C082E50B
:100BA0008093C10081E08093C70018BC19BC7AC053
:100BB0008091BC008430A1F480916300882381F08F
:100BC0001092CC001092DF001092C1009091C600EC
:100BD00081E0282F291B2093C6008093C70062C0A4
:100BE0008091C60081115EC08091BC00833041F4C9
:100BF00080E58093C10081E08093C70018BC19BCD8
:100C00008091BC00823071F48091A6008F3F11F476
:100C100041DB48C086E98093CC008091CC00809372
:100C2000DF0035C08091C70081113CC08091CC00AD
:100C300081111AC08091C800811103C081E08093A6
:100C4000C80081E08093C90092E09093CA0090911F
:100C5000C8009093CC009093DF009091640099239A
:100C600039F08093AD0004C01092CC001092DF00E8
:100C70008091DF008F3F59F480916A0018BC89BDD4
:100C80008091EB00882371F080E0C5DA0BC0F6DAC2
:100C900009C01092BC0080916400882319F081E0A3
:100CA0008093AD001092C70098C02831310508F03C
:100CB00078C08091C100803509F44BC08091C1009B
:100CC000813509F446C08091C100823509F441C0E4
:100CD0008091C100811106C08091BC00811102C0C9
:100CE00081E007C08091BC00882329F08091BC007E
:100CF0008F5F8093BC008091C60081116EC080918F
:100D0000CF00882379F08091BB00882359F080912F
:100D1000C100811107C08091BB008093C100109277
:100D2000BB005BC08091C1008031F0F48091C100B4
:100D3000882391F08091B9009091BA008B3491058D
:100D400058F08091C1008093BB008091C1008093D6
:100D5000C0001092C10041C08091D000882311F0E2
:100D6000B6DB3BC0A0DB39C08091B9009091BA00DE
:100D70008B34910510F09BDA30C08091680081308F
:100D8000D1F3E091F000EF5FE093F00080916C0010
:100D9000E81788F7F0E0E356FF4F80818093C100A9
:100DA0001CC024343105B8F48091BC00813099F422
:100DB0002091B9003091BA002E30310560F4909145
:100DC000C100911108C09091EB00891B8093EB004A
:100DD0008091EB0020DA1092BC001092BA001092C1
:100DE000B900D2C08091B9009091BA000196909359
:100DF000BA008093B900892B31F480E395E7909392
:100E0000BA008093B9008091B9009091BA000F9711
:100E100010F01092BC00809169008230E8F180915E
:100E20006B008823E1F08091DF0084578B38A0F5B8
:100E30008091A7009091A80001969093A8008093BC
:100E4000A7002091B7003091B8002817390720F586
:100E500086E68093CC008093DF00EBD91DC08091A3
:100E6000C1008031C8F4E091C100F0E0E052FF4FD2
:100E700080818F3F89F48091A7009091A80001960E
:100E80009093A8008093A7002091B7003091B800FC
:100E90002817390708F41BDB80916B00882391F039
:100EA0008091CC00823070F08091CC00863950F473
:100EB0008091B9009091BA008C34910518F081E0CE
:100EC0008093C9008091600090916100009729F0A3
:100ED00001979093610080936000809160009091F1
:100EE0006100892BD1F59091C10080916B00811137
:100EF00004C081E0913041F408C09091DF0081E0AE
:100F0000913019F09F3F09F080E02091B20030E06D
:100F1000811103C080E290E002C08EE190E02817CA
:100F2000390734F48091A5008F5F8093A50004C039
:100F30001092A5001092B4008091A500883068F04E
:100F400081E08093B5008093B4001092A50088E3FF
:100F500091E090936100809360008091B4008823B9
:100F600099F08091A3009091A40001969093A40021
:100F70008093A300843F914039F481E08093B300D3
:100F80001092A4001092A3001092BE001092BD0017
:100F90008091A2008F5F8093A200837019F486B1C4
:100FA000886486B9FF91EF91BF91AF919F918F9126
:100FB0007F916F915F914F913F912F910F900FBE55
:100FC0000F901F901895CF93DF931F92CDB7DEB788
:100FD00017BA88E088BB85BB83E087BB81EA8ABDFE
:100FE00081E083BF8CE087B9A29A87EC86B9479AE3
:100FF00085B7877E806185BFF8948BB78F7D8BBF67
:10100000A89584B7877F84BF81B5886181BD11BCF5
:101010001092AC001092AB000091AB001091AC00AC
:101020000038110508F05EC6C80194D6F82E8093EA
:10103000EF00C80101968ED6E82E8093DB00C80130
:10104000029688D6D82E8093ED00C801039682D6EA
:101050008D3539F00C5F1F4F1093AC000093AB003F
:10106000DBCF8F2D87708093C1008F2D869586955D
:1010700086958F7080936700FF1CFF24FF1CF09201
:101080006B008E2D81708093D000E1FA882780F963
:101090008093CF008E2D86958695877080936A0009
:1010A000E294E69487E0E822E09269008D2D817059
:1010B0008093CD00D1FA882780F980936400D2FA1A
:1010C000882780F980936500D3FA882780F9809378
:1010D000CE00D4FA882780F9809366008D2D829502
:1010E0008695837080936800809165008093EB0003
:1010F0008AEF90E02FD69FEF980F9E3F10F48093D9
:101100006200E0916700F0E0E45CFF4F849180931F
:10111000DD001092D1001092E000909166009923BA
:1011200041F01092E10090916A009093D20092E019
:1011300001C091E020E030E0482F50E0692F70E0DE
:101140002417350734F5A0916700B0E0AA0FBB1F44
:10115000AB57BF4FED91FC91E20FF31FE491890172
:10116000060F171FD801A052BF4FEC93A091670044
:10117000B0E0AA0FBB1FA359BF4FED91FC91E20F46
:10118000F31FE491D801AF52BF4FEC932F5F3F4F55
:10119000D7CF890F8093DD00E0916900F0E0EE0F7A
:1011A000FF1FE45DFF4F859194919093B800809369
:1011B000B7008091CD00882359F080916B00811198
:1011C00007C08091F100811105C06DD99BD902C083
:1011D0001092C1008091C100811104C060E570E0EF
:1011E00082E077D81092F1008AEF8093EC0089E1D9
:1011F0008093EE00F894A89581B5886181BD80E464
:1012000081BD7894A12C912C55245394AFE04A2EA3
:10121000BB24BA94B8E3EB2EFF24F3940CEF1AE04E
:1012200085E0C82ED12C88248A948091C500811134
:1012300072C28091C6009816C1F09090C60018BC8A
:1012400019BC8AEF90E0DED76CE370E084E041D80F
:101250001092C7008091C600882329F08091C100B8
:101260008093EC0002C08092EC009091C1008091CC
:10127000EC00981709F404C18091C100803140F559
:101280002091C100822F90E0FC01E052FF4F30819D
:101290003093DE00FC01EF52FF4F80818093DC0031
:1012A0008091DC009091DE0098BD89BD211106C0BF
:1012B0008091EB00882311F081E004C08091EC0064
:1012C000811101C0A8D78091C1008093EC00D8C0E3
:1012D0008091C1008093EC0019BC18BC8091C100C2
:1012E000803579F480E991E08DD71092C700809124
:1012F000C100803509F0C4C08091B20060E53AD8E1
:10130000F6CF8091C100813579F48AEF90E07AD7E9
:101310001092C7008091C100813509F0B1C0809161
:10132000B10061E527D8F6CF8091C100823571F414
:101330008AEF90E067D71092C7008091C100823594
:1013400009F09EC062E58DE015D8F7CF8091C1000D
:101350008B3549F48091C1008B3509F091C06FE263
:1013600080E17AD7F7CF8091C1008C3501F580916B
:10137000C1008C3509F084C0F8E07F2E8091C10057
:101380008C3519F0E8E07E2E0DC068E284E164D768
:101390007A947110F3CFF6CF60E588E25DD77A9446
:1013A000772029F38091C1008C35B1F3E0CF809193
:1013B000C1008D3549F58091C1008D3511F574E07E
:1013C000772E8091C1008D3519F06AE0762E14C019
:1013D000B8BC19BC85E090E015D718BCB9BC81E455
:1013E00090E010D77A947110ECCFEFCF88E490E0C2
:1013F00009D77A947720F9F28091C1008D35B1F345
:10140000DACF18BC19BC3CC08091C1008E35D1F434
:101410008091C1008E35A1F58CE291E0F3D66DE7A5
:101420008DE71AD76DE78DE717D75FE0752E8091AE
:10143000C1008E3569F784E690E0E4D67A947110A5
:10144000F6CFE6CF8091C1008F35D1F48091C100F5
:101450008F35B1F48CE291E0D5D660EF80EFFCD609
:1014600060EF80EFF9D644E6742E8091C1008F358D
:1014700069F784E690E0C6D67A947110F6CFE6CF8D
:101480008091B500882309F445C080916B008823C2
:1014900069F18091DF008823D1F1813011F08F3F15
:1014A00061F487E08093DF0088E085D71092CC005C
:1014B0001092DF001092CB0012C083E07CD78091A5
:1014C000DF008A3050F090E0880F991F880F991F35
:1014D000B6012DD46093DF0002C05092DF008091EE
:1014E000DF00CCD68AEF90E08DD611C08091C1008C
:1014F000882369F08091C100813011F488E001C037
:1015000083E059D78091C100803108F4E0D7109270
:10151000B50028C08091B300882321F18091640038
:101520008823F1F08091C100811104C08091EB000B
:10153000811105C062E084EF91E06FD711C080E0B7
:101540006AD684EF91E05ED681E065D684EF91E0C3
:1015500059D680E060D684EF91E054D681E05BD626
:101560001092B300809169008130B9F59091B1007B
:1015700080916200981788F18091AE009091AF0041
:10158000892B59F580916B008823B1F08091DF00A1
:10159000823418F1282F30E066E0A9D3A901481B56
:1015A0005109CA01423451050CF481E48093DF00F3
:1015B0008091DF0063D609C08091C100882369F063
:1015C0008091C100803148F482D71093AF0000931E
:1015D000AE0063E084EF91E020D78091B4008823CF
:1015E00029F024EE622E27E5722E04C096E3692EC0
:1015F0007724739480916B00811104C08091C100A5
:10160000882349F080916B00882309F45AC08091A7
:10161000DF00811156C02ED7892B09F052C080916E
:10162000B9009091BA006816790608F04AC0809116
:10163000B200803230F48091EB00882311F080E01A
:10164000EAD581E090E0DED51092BA001092B900A0
:101650001092AF001092AE00F894A89584B7877FDF
:1016600084BF81B5886181BD11BC78943798109290
:10167000BE001092BD00FED6892B21F080E190E0E3
:10168000C1D5F9CF8BB780628BBF85B7806285BF2C
:1016900085B7846885BF8B7F85BF889585B78F7D2B
:1016A00085BF8BB78F7D8BBF8CE087B9A29A87EC03
:1016B00086B9F894A89581B5886181BD80E481BD23
:1016C00078948091AD00882309F4AFCD8091DF003C
:1016D000811103C01092AD00A8CD82548D3B10F44F
:1016E00022E001C021E08CE291E029838BD52981A1
:1016F00081E0298390D58FEA90E084D580E08BD576
:101700002981223029F48FEA90E07CD521E0F0CFC6
:101710002130E1F7DFCF8091C3008A1571F0A090EE
:10172000C3008091C300882341F018BC84E189BDC7
:1017300084E690E067D518BC19BC9091C5008091F3
:10174000C400981709F4B2C28091C5008093C40008
:101750001092C2008091C500883109F46DC078F400
:101760008F30C9F128F48130E1F0833019F1C2C023
:10177000853109F445C0873109F44FC0BBC08932B7
:1017800009F48DC038F4893109F463C0883209F452
:101790008AC2B0C0843609F468C0853609F470C0C6
:1017A000A9C080E991E02ED581E053D68091C50093
:1017B0008F5F62C28091C300882359F08091C3007B
:1017C000893038F48091C3008170852580936B0047
:1017D00099D682E0DAC11092C50068E270E085E037
:1017E00078D51092CC001092DF001092C100809149
:1017F0006B00882309F457C28091CC003FD553C2B7
:1018000080E991E0FFD481E024D68091C5008F5F0C
:101810008093C5001092C30046C28091C300882304
:10182000C1F28091C300817085258093650080910D
:1018300065008093EB00CCCF8091C300882339F002
:101840008091C300817085258093CE005BD683E0B4
:101850009CC18091C300882309F423C28091C300F6
:1018600081708525809364001BC268E270E083E08C
:1018700030D5B8BC19BCF092AF00E092AE0013C2F4
:1018800018BC19BC8091AE009091AF00892B11F566
:101890006091B100609362008AEF2BD61BC08091EB
:1018A000C3008823B9F08091C300873098F48091F9
:1018B000C3008F5F8093690025D6E0916900F0E056
:1018C000EE0FFF1FE45DFF4F859194919093B80058
:1018D0008093B70080916B00882321F084E0B9D514
:1018E00085E003C088E0B5D589E08093C50080938A
:1018F000C400D9C180916B00882309F47FC0809116
:10190000C500853009F45EC0863009F474C08430A7
:1019100009F0C9C18091C300882309F498CF809150
:10192000C300883008F093CF8091C30080936A0091
:10193000E0916700F0E0E45CFF4FA491A093DD002C
:101940001092D1001092E00080916600882341F04F
:101950001092E10080916A008093D200B2E001C051
:10196000B1E080E090E04A2F50E06B2F70E08417E8
:1019700095070CF0A8C0E0916700F0E0EE0FFF1FA4
:10198000EB57FF4F0190F081E02DE80FF91F7490A5
:101990009C01260F371FF901E052FF4F7082E09142
:1019A0006700F0E0EE0FFF1FE359FF4F0190F08159
:1019B000E02DE80FF91F74902F523F4FF90170820C
:1019C0000196D5CF8091C300813019F4109269003F
:1019D000D0C08091C300823019F4509269004AC18E
:1019E0008091C300833029F468E270E04BC181111B
:1019F0006EC084E0CAC08091C30047C1E091C500B9
:101A00008E2F90E0FC013497E730F10508F04BC1D0
:101A1000E15FFF4F8091C3000994882309F417CF39
:101A20008091C3008D3008F012CF8091C3008150A7
:101A300080936700E0916700F0E0E45CFF4FA491C1
:101A4000A093DD001092D1001092E000809166001A
:101A5000882341F01092E10080916A008093D200C7
:101A6000B2E001C0B1E080E090E04A2F50E06B2F7F
:101A700070E0841795073CF5E0916700F0E0EE0F09
:101A8000FF1FEB57FF4F0190F081E02DE80FF91F8A
:101A900074909C01260F371FF901E052FF4F7082AE
:101AA000E0916700F0E0EE0FFF1FE359FF4F019058
:101AB000F081E02DE80FF91F74902F523F4FF9018C
:101AC00070820196D6CFAB0FA093DD00BFCE809180
:101AD000C3008170852580936600E0916700F0E087
:101AE000E45CFF4FA491A093DD001092D10010920E
:101AF000E00080916600882341F01092E10080911F
:101B00006A008093D200B2E001C0B1E080E090E0D2
:101B10004A2F50E06B2F70E0841795073CF5E09159
:101B20006700F0E0EE0FFF1FEB57FF4F0190F081D1
:101B3000E02DE80FF91F74909C01260F371FF90163
:101B4000E052FF4F7082E0916700F0E0EE0FFF1F60
:101B5000E359FF4F0190F081E02DE80FF91F7490D9
:101B60002F523F4FF90170820196D6CFAB0FA09351
:101B7000DD00C8D43ECF882339F08091C300817046
:101B800085258093D000BED485E063D48CC08823A3
:101B900039F08091C300817085258093CF00B2D445
:101BA00086E0F3CF882309F456C08091C3008830C3
:101BB00008F051C08091C30080936A00E0916700F3
:101BC000F0E0E45CFF4FA491A093DD001092D100FF
:101BD0001092E00080916600882341F01092E100AD
:101BE00080916A008093D200B2E001C0B1E080E051
:101BF00090E04A2F50E06B2F70E0841795073CF57A
:101C0000E0916700F0E0EE0FFF1FEB57FF4F0190F0
:101C1000F081E02DE80FF91F74909C01260F371F0B
:101C2000F901E052FF4F7082E0916700F0E0EE0FA3
:101C3000FF1FE359FF4F0190F081E02DE80FF91FDE
:101C400074902F523F4FF90170820196D6CFAB0F9F
:101C5000A093DD0057D487E098CF811105C0109282
:101C6000690050D488E091CF8091C300813039F46D
:101C70008093690047D484E68093C50014C068E26D
:101C800070E083E026D388E2F7CF882351F080917B
:101C9000C300843030F48091C30081508093680089
:101CA00031D44092C5001092C300BFCA8091C300D6
:101CB000882321F08091C2008F3370F48091C50099
:101CC000843609F4B2CA8091C3008111AECA8091F2
:101CD000C200893C08F4A9CA8091C5008F5F809337
:101CE000C500A3CA1092AC001092AB00FDC9991BAD
:101CF00079E004C0991F961708F0961B881F7A9503
:101D0000C9F780950895AA1BBB1B51E107C0AA1F04
:101D1000BB1FA617B70710F0A61BB70B881F991F8C
:101D20005A95A9F780959095BC01CD01089597FB30
:101D3000072E16F4009406D077FD08D0E4DF07FCE8
:101D400005D03EF4909581959F4F089570956195CB
:101D50007F4F0895E199FECF9FBB8EBBE09A9927F4
:081D60008DB30895F894FFCF44
:101D6800380134010101010302050301059E009AAF
:101D78000094008C0082007600680062005C0056C7
:101D880000500048009F009C009700900087007C4E
:101D9800006F0065005F00590053004C005B5C5DFC
:021DA8005E5F7C
:00000001FF
